:02000000806F0F
:06000B00C2AFC28C804769
:10002300C2AFC0D0C0E01098051099208020C2B79D
:100033007A0A307E04E5998015A699B83F04743096
:100043008002E804B501028005F88002C27FD0E097
:10005300D0D0D2AF32BC000280011CBA0004D2B7A8
:1000630080011A758AF0758CD8D2AFD28C32758123
:10007300503160D2B77A00C27E78307930758AF019
:10008300758CD8759850758DFF7589217588507555
:10009300A89231A8312C11B111CF207EF911ED6056
:1000A300F530F70474203131E5F03106019920B1C0
:1000B3001AC2AF7C05D2AFBC00FD20B10E30B1FD3A
:1000C300C2AF7C05D2AFBC00FD312C2220B21AC2D4
:1000D300AF7C05D2AFBC00FD20B20E30B2FDC2AF83
:1000E3007C05D2AFBC00FDB27E22C2AFE8B50102EF
:1000F300800C87F07401B93F02792F0980027400E4
:10010300D2AF22F5F0E5F0C4540F311A3131E5F0E6
:10011300540F311A313122C0E0C3940A5006D0E0A3
:1001230024308004D0E02437227401314222F59038
:10013300C2B3D2B500D2B400C2B4C2B5318D22F578
:1001430090C2B3C2B5D2B400C2B4318D2275F008E7
:10015300A4FF7E007DFFDDFEDEFCDFFA22C2B3C218
:10016300B5C2B4759000740F319B7E04759038D27C
:10017300B4C2B47404319BDEF6740E314274073199
:1001830042741831427401314222D2B3D2B4D297AD
:100193002097FDC2B4C2B3227FEC00000000DFFA57
:1001A30000D5E0F4229001B9E49360053131A380D6
:1001B300F774043150225365654D696469205631E3
:1001C3002E3020202020202020202020202020200E
:1001D3002020202020202020202020202020436FAA
:1001E3007079726967687420544D4420496E6E6F4C
:1001F300766174696F6E7320323030362020202090
:070203002020202020200034
:00000001FF
